:0A05F900C0F9A4B0999282F8809036
:0C05EC00010A00011100041300000000CF
:10054B00E4F517F50CF50BF518F50EF50D750D1704
:10055B00750E3B751837F50BF50C75171EF51975E0
:0B056B000801F50FF510F512F509224C
:040576007F147E0070
:10057A00E4FDFCC3ED9FEC9E5015E4FBFA0BBB00B7
:0F058A00010AEB646E4A70F50DBD00010C80E4B0
:01059900223F
:1005B000758911758CD8758AF0D2AFD2A9D28C22E8
:1005C000758911758D3C758BB0D2AFD2ABD28E22AE
:0D05DF00D2AFD2A8D288D2AAD28AD2B92235
:03000B00020514D7
:10051400C0E0C0D0758CD8758AF00511E511B464BB
:10052400217511000518E518B43C17751800050E5F
:10053400E50EB43C0D750E00050DE50DB4180375FC
:070544000D00D0D0D0E03221
:03001B000203E5F8
:1003E500C0E0C0F0C083C082C0D075D000C000C0DE
:1003F50001C002C003C004C005C006C007758D3C1E
:10040500758BB0E4FAF9F8E5162401F516EA351509
:10041500F515E93514F514E83513F513E47F14FEE5
:10042500FDFCAB16AA15A914A813C312059A7026CC
:10043500F516F515F514F5130509E509B43C177519
:1004450009000512E512B43C0D7512000510E51002
:10045500B41803751000E510B5190AE512B50805BD
:10046500750A018003750A00D007D006D005D004AF
:10047500D003D002D001D000D0D0D082D083D0F02C
:03048500D0E03292
:0300030002001EDA
:10001E00C0E0C0F0C083C082C0D075D000C000C0A8
:0D002E0001C002C003C004C005C006C00729
:10003B00751A20751B00751C00751D00751E00754B
:10004B001A20E4F9751C00E97004E50F801AB90158
:10005B0004E50F8024B90204E508800CB90304E51C
:10006B00088016B9040EE51975F00A8485F01B7526
:10007B001C018010B9050AE51975F00A84F51B807F
:10008B0003751BFF7580FFE51CB4010CE51B900588
:10009B00F9936480F51F8008E51B9005F993F51F14
:1000AB00E9C313B51D1C051EE51EB4C803751E0060
:1000BB00E51EC39400400BE51E94645005751FFFAD
:1000CB008000851F80851AA0AF1A7801EF08800188
:1000DB0003D8FDF51A7F027E0012057A09E9640642
:1000EB00600302004FC29620900B120576209005FC
:1000FB001205C0807320911312057620910D051DFA
:10010B00E51DB40303751D003091FD309203020011
:10011B004A12057630920302004AE51D7020050F46
:10012B00E50F643C703AF50F0508E508643C703048
:10013B00F5080519E51964187026F5198022E51DD7
:10014B00B401130508E508B43C167508000519E55C
:10015B0019B4180C80070519E519B41803751900A3
:08016B0030920302004A80F803
:10017300D007D006D005D004D003D002D001D000E0
:0B018300D0D0D082D083D0F0D0E0328A
:0300130002018E59
:10018E00C0E0C0F0C083C082C0D075D000C000C037
:0D019E0001C002C003C004C005C006C007B8
:1001AB0075202075210075220075230075240075BC
:1001BB002020E4F9752200E97004E517801AB901D3
:1001CB0004E5178024B90204E50C800CB90304E59F
:1001DB000C8016B9040EE50B75F00A8485F02175B9
:1001EB0022018010B9050AE50B75F00A84F5218010
:1001FB00037521FF7580FFE522B4010CE521900505
:10020B00F9936480F5258008E5219005F993F52590
:10021B00E9C313B5231C0524E524B4C803752400D6
:10022B00E524C39400400BE524946450057525FF29
:10023B0080008525808520A0AF207801EF08800104
:10024B0003D8FDF5207F027E0012057A09E96406CA
:10025B0060030201BFC296209006120576309073A0
:10026B0020911312057620910D0523E523B403038A
:10027B007523003091FD3092030201BA12057630DE
:10028B0092030201BAE52370200517E517643C7051
:10029B003AF517050CE50C643C7030F50C050BE5D5
:1002AB000B64187026F50B8022E523B40113050CA3
:1002BB00E50CB43C16750C00050BE50BB4180C8063
:1002CB0007050BE50BB41803750B00309203020105
:0302DB00BA80F8EE
:1002DE00D007D006D005D004D003D002D001D00074
:0B02EE00D0D0D082D083D0F0D0E0321E
:1002F900752620E4F527F528F529F52AD2967526DD
:1003090020E4F9E4F528E97004E518801AB9010434
:10031900E5188024B90204E50E800CB90304E50E42
:100329008016B9040EE50D75F00A8485F027752845
:10033900018010B9050AE50D75F00A84F5278003D7
:100349007527FF7580FFE528B4010CE5279005F9AD
:10035900936480F5808008E5279005F993F58085F9
:1003690026A0AF267801EF08800103D8FDF5267F86
:10037900027E0012057A09E964067087E52970048E
:10038900D297801D052AE52AB41403E4F52AE52A43
:10039900C39400400AE52A94055004C2978002D20A
:1003A90097E529701FE50DB50B0BE50EB50C06E5B4
:1003B9001865176009E50A640160030203057529D8
:1003C90001020305309009309106309203020305BA
:0C03D900E4F5297F14FE12057A020305EA
:0F05D00012054B1205B01205DF1205760202F973
:030000000204886F
:0C048800787FE4F6D8FD75812A0204CFCD
:10059A00EB9FF5F0EA9E42F0E99D42F0EC6480C8D8
:0605AA0064809845F02278
:100494000205D0E493A3F8E493A34003F68001F2A9
:1004A40008DFF48029E493A3F85407240CC8C33369
:1004B400C4540F4420C8834004F456800146F6DF38
:1004C400E4800B01020408102040809005ECE47ED7
:1004D400019360BCA3FF543F30E509541FFEE4932D
:1004E400A360010ECF54C025E060A840B8E493A3F4
:1004F400FAE493A3F8E493A3C8C582C8CAC583CA1F
:10050400F0A3C8C582C8CAC583CADFE9DEE780BED6
:0105F8000002
:00000001FF
